:020000040000FA
:1000000007309F00003083169F0186008500831211
:1000100040201D20282034200F2071200A283F3046
:1000200084001030A4000008840A80008403840344
:10003000A40B13284008B0000800303084001030B2
:10004000A400240875208000840AA40B212808003D
:10005000803049200830A3003F308400000855203C
:100060008403A30B2E280800C03049200830A300C9
:1000700037308400000855208403A30B3A28080079
:100080003830492001304920033049200F304920C1
:100090000800860061200430850061200030850062
:1000A0006120043085006120080086006120063050
:1000B00085006120023085006120063085006120C6
:1000C00008000A30A200A100A10B6428A20B63283B
:1000D0000800FA30A200A100A10B6C28A20B6B282B
:1000E000080069206920692008008207203445340F
:1000F0004434553450344934433420343134363464
:0E01000046343634323438342E342E342E3415
:02400E00293F48
:00000001FF
